:030000000219FDE5
:03000B000200AA46
:03002B0002015679
:03005B000202E5B9
:030073000202D2B4
:1000800002030406080C10182030406080040608A3
:100090000C10182030406080A0C00003070F1F0D17
:1000A0000D0403060D0502030202C2AFC0D0C0E07A
:1000B000206214E5256009E473E525F4F58AD2622F
:1000C000D0E0D0D0D2AF3285268AC262E526F46075
:1000D00029D0E0D0D0D297D295D293D2AF32D29756
:1000E000D295D293206F0C2066097405D5E0FDE50A
:1000F0007B4290D0E0D0D0D2AF32758A00C28DD290
:100100006201F301B9306805206602C29701B93077
:100110006805206602C29301B9306805206602C2F4
:100120009501B9C29630680A206607740FD5E0FDC4
:10013000C29701B9C29230680A206607740FD5E0F1
:10014000FDC29301B9C29430680A206607740FD5C6
:10015000E0FDC29501B9C2AFC2AD53E6EFC0D0C059
:10016000E0D2D3D2AFC2CEE52A6007207449152A67
:1001700021B77800790020742EE580307E01F430BC
:10018000E50278FF53DACF207E0343DA20307E0386
:1001900043DA10C2D8C271E580307E01F430E50246
:1001A00079FFC3E89970CB306103752A402074034E
:1001B000752A40885CD27020740DE52B6004152BE5
:1001C00021C743DA01C2D820700221DAA85C20617D
:1001D00002C27020740221D888227882B604038576
:1001E0002224C3E52594404002D26420CF0AD0E007
:1001F000D0D043E610D2AD32C2CF053A7802E52A1C
:100200006005307402152AC3E55C94014005755FF2
:10021000004124756000756900E55F2401F55F50B9
:1002200003755FFF7982B7020D306E1DC3E522941E
:10023000324016854C227982B7030E306E0BC3E52F
:100240002294324004798E8722C3E52395226008E8
:100250004004152341580523D8CA0569E569700291
:100260001569D56A63756A017805C3E569956B40C0
:1002700057C3E569956C50087801756A0302028CD2
:10028000C3E569956D50057801756A01C3E562950E
:1002900024401E7982B7040241BD206E1485246279
:1002A000E569046003856B69756A0175233C020288
:1002B000C8E5622850057562FF41BDF562E562043C
:1002C00070067560FF7569FFD0E0D0D043E610D2AC
:1002D000AD32C2AF53E67F7592FA7593FFC2607577
:1002E0009104D2AF32C2AF53E6EFC2ADC0D0C0E08E
:1002F000C0F0D2D3D2AFA8FBA9FCC2D83071026142
:100300004C53DACF207E0343DA10307E0343DA20E9
:10031000D271E580307E01F420E5026123882789CF
:1003200028A13153DACF207E0343DA20307E034305
:10033000DA10C2D8C271307402A11D7800E5803095
:100340007E01F430E502A11D885CA10553DACF20BF
:100350007E0343DA20307E0343DA10C2712061024B
:10036000812553DACF207E0343DA10307E0343DA4F
:1003700020C2D8D27188578958C3E89555F8E995B5
:1003800056F97B007E087A00C3E8948CE99400500B
:1003900005755B008117882178A2E6A8216055C306
:1003A000E894C8E994005008E4D2E4FB7A0A61F2C8
:1003B000C3E89468E994015008E4D2E3FB7A0F6142
:1003C000F2C3E894D0E994025008E4D2E2FB7A1E2A
:1003D00061F2C3E894A0E994055008E4D2E1FB7A05
:1003E0003C61F2C3E89498E994085008E4D2E0FB39
:1003F0007A787E00C3E89559FCE9955AFD30E70A02
:10040000ECF42401FCEDF43400FD755B00C3EC9AC0
:10041000ED9E5003755B018859895A85575585585B
:10042000567802A105C3E89527F8E99528F9307CAC
:100430000281E9307B0281E9307A0281E220750293
:100440008148E9FDE8FC8167E9C313F9E813F83056
:10045000790281E2E9C313F9E813F830780281E206
:10046000E9C313FDE813FC20612CC3EC941CED944C
:0E047000024002817EED701EC3EC94C850184D
:10047E000529E52970021529C3E529940A5002A120
:10048E001D755C00D270A11DE5296002152974004E
:10049E00207F037896E624FAFEE43400FFC3EC9E38
:1004AE00FCED9FFD50067800790081E9C3EC94FFC6
:1004BE00ED9400400678FF790081E9EC8572F0A496
:1004CE00C5F0A2F733F87900400302050578FF79ED
:1004DE0000020505E9C313F9E813F8307C0EE96054
:1004EE000278FFC3E81338F8E43400F9C3E894FF48
:1004FE00E99400400278FF885CD270206102A11D51
:10050E00741FF4552F4BF52FC274EB7002D2747515
:10051E002A40307403752A0A306102A13120740317
:10052E0053DAFE207403752B20D0F0D0E0D0D0D259
:10053E00AD43E61032790102056179030205617956
:10054E000A020561791E020561796402056179C8A6
:10055E000205617817E4D5E0FDD8FAD9F6227A14AF
:10056E007B780205887A107B8C0205887A0D7BB425
:10057E000205887A0B7BC80205887902E4C292D5FF
:10058E00E0FDC293D5E0FDD293D5E0FDD292D5E049
:10059E00FDE920E002C29730E002C295E573D5E096
:1005AE00FDE920E002D29730E002D2957496D5E0B4
:1005BE00FDD9C9EAF8D5E0FDD8FBDBBEC29222C355
:1005CE007C007D0075F00005F0EA33FAEB33FB504A
:1005DE00F6EB13FBEA13FAC3E9FFE8FEE89AF8E933
:1005EE009BF95004EFF9EEF8B3EC33FCED33FDD587
:1005FE00F0DFEDF9ECF822E889F08A20D2D4F8A9E0
:10060E00F07B0030F70B7BFFF42401F8E9F43400A3
:10061E00F9E88520F0A4ADF0F8E98520F0A4AFF05C
:10062E00FEED2EF974003FFA7C04C3EA13FAE913C7
:10063E00F9E813F8DCF48BF030F70AE8F42401F84B
:10064E00E9F43400F9E889F0C2D4F8A9F0227882EE
:10065E00B604030206FBC3E55C9419401EE52D5457
:10066E00067018206E3678057994E7146007780ABC
:10067E001460027812C3E54198401F306E098564FC
:10068E00627569FF756A01852224E4F544F545F526
:10069E0046F547F548C26E0206FBD26E7994E71412
:1006AE007013E523F43333F913F8E9540104F9E830
:1006BE0054FE0206EFE714147014E523F4333333BB
:1006CE00F913F8E9540304F9E854FC0206F7E5239C
:1006DE00F433333333F913F8E954070404F9E854C7
:1006EE00F8C39440F8E99400F98844894522C3E59B
:1006FE004113F9E54013F8C3E54498F8E54599F937
:10070E00500CC3E89480E994FF4016020733C3E807
:10071E00947FE994005003020733787F7900020733
:10072E0033788079FF8849894A22E5492546F8E5DC
:10073E004A3547F9854A20E4300701F43548FA3046
:10074E00E709C3EA94F04015020771C3EA940F500B
:10075E000302077178FF79FF7A0F0207717800792B
:10076E00007AF0C3E5249561500AC37401952450B4
:10077E000B02078FE54A20E70E02078FE54A30E7A6
:10078E0006884689478A482278A5E6FAC3E54933A2
:10079E00F8E54A33F9D105E930E70BC3E89480E96F
:1007AE0094FF4013E1C9C3E8947FE994005002E13D
:1007BE00C9787F7900E1C9788079FFE820E715C311
:1007CE00E52398F84009C3E8940140030207F07846
:1007DE00010207F0E8F424012523F840030207F094
:1007EE0078FF884B2278A6E6FAA847A948D105E9F2
:1007FE0030E70CC3E89401E994FF4016020824C3C5
:10080E00E894FFE99400500302082478FF7900026F
:10081E000824780179FFE920E715C3E54B98F840E5
:10082E0009C3E89401400302084B780102084BE823
:10083E00F42401254BF8400302084B78FF8824224C
:10084E0078FFC26420693D206A12D264C3E54194E8
:10085E000A4009C3E52594405002C26479A1E760BD
:0E086E0023E541601F74FF8541F0848539F059
:10087C00306A0375F005A4F8C5F0600278FFC3E890
:10088C0095645002A864886322C3E5409440E54116
:10089C009401E56350031401A6046002F563227809
:1008AC0083E6F520120F2275E89012054375E89047
:1008BC00E5E820ECFBA8BDA9BE120FC8756E5575F6
:1008CC006F00C3740013FD7455606613FC74552CD3
:1008DC00FC74003DFDECFAEDFBC3E89AE99B401477
:1008EC00E56E2455F56EE56F3400F56FEA2CFAEBE6
:1008FC003DFB80E5AE6EAF6FC3E56F13F9E56E138C
:10090C00F8C3E913F9E813F87A03C3E913F9E81308
:10091C00F8DAF7AA201A7009756E00756F000209D3
:10092C003D1AEA6008EE28FEEF39FFDAF88E6E8F7A
:10093C006F2275E890227883E6FFE5E820ECF7A8B3
:10094C00BDA9BE0570C3E57094084052757000E9EE
:10095C00FA79A0E76044EA7007E571601B02097838
:10096C00C3E895716010E5715006600C140209849F
:10097C000460F9020984E571F571C3946D401B752F
:10098C0061C0C394044013756180C39404400B751B
:10099C006140C39404400375610075BB0822EFC32A
:1009AC009401601F7455601BC3E894FFE9940350D5
:1009BC0012C3E8956EE9956F5009E561600C1561FD
:1009CC000209D6E561F460020561A861C3E52498CB
:1009DC005002A824C3E89562400AA862E562F4605C
:1009EC000385626188258826E570B4070375BB1002
:1009FC0022743279A787F0A4C5F0A2F733F8C3E8C4
:100A0C0095614002A86188228824882588268864FC
:100A1C00227540007541F022C2AF75C820A8CCA940
:100A2C00CDAA3A30CF010A75C824D2AFAB3BAC3C4F
:100A3C00883B893CC3E89BF8E99C206908F930673E
:100A4C00026130418DAD3D8A3DF9EA9DFA60047832
:100A5C00FF79FFAE3EAF3F8B3E8C3FA83BA93CC31A
:100A6C00E89EF8E99FF9C3E54113FBE54013FAE86A
:100A7C002AF540E93BF54150067540FF7541FF41B1
:100A8C00D7AA40AB41AC40AD417E047F02C3EB948E
:100A9C000440021E1FC3EB940840021E1FC3ED133B
:100AAC00FDEC13FCDEF7C3EA9CFAEB9DFBEF60094F
:100ABC00C3E913F9E813F8DFF7EA28FAEB39FB8AF4
:100ACC00408B4150067BFF8B408B41C3EB94025013
:100ADC0002D2673069047F0361027892E6FFC3E5B6
:100AEC0037948240110FC3E53794A040010FC3EF38
:100AFC00940640027F057E02E541C4540FF9E5419E
:100B0C00C454F0F8E540C4540F28F8C3E89EFAE941
:100B1C009400FB4009C3EA9402EB940050047A025F
:100B2C00E4FB617CAA40AB41EBC4FEEAC4540F4E1B
:100B3C00FCC3EA9CFAEB9400FBC3E813C313F8EA7A
:100B4C0028FAEB3400FB8A408B41C3EB9402400241
:100B5C00C2677802EBC4FE7B00EAC4540F4EFAC3A2
:100B6C00EA98FA4005C3940250027A027892E6FFA2
:100B7C00306002617C855192855293D26043E6804D
:100B8C00C3E49AF8E49BF93067028108E8FAE9FBC0
:100B9C00D3E913FDE813FC88518952C3EF94036029
:100BAC0038EF20E00DE82CF8E93DF9ECFAEDFB020A
:100BBC000BD1E828F8E939F9C3E82402F8E9340044
:100BCC00F97AFE7BFFC3EF9403400E8A538B548853
:100BDC004D894E8C4F8D50813C885389548A4D8B56
:100BEC004E8C4F8D503069127553F07554FF754F04
:100BFC00F07550FF7551F07552FF813CE8FAD3E85F
:100C0C0013FC8851C3EF94036020EF20E007E82C1D
:100C1C00F8ECFA8128E8282402F87AFEC3EF940352
:100C2C0040088A53884D8C4F813C88538A4D8C4F99
:100C3C00E568C3335002646BF56830600281467519
:100C4C003402D26043E680E52D54066034A840A9F6
:100C5C0041C3E913F9E813F8C3E913F9E813F830C1
:0F0C6C006904E92440F9C2AF53E67F759100C3D4
:100C7B00E498F594E499F595759104D26043E68078
:100C8B00D2AF22D265754300752000306C037520FE
:100C9B0040020CADD265754300752040306C037576
:100CAB00200078017901206720E52D54066002C2EF
:100CBB00657914E541C313700104F8C39414400221
:100CCB007814306904781B791B206010E543600CA5
:100CDB00306903D53404D26DA14F914E0543E59B8A
:100CEB005440B52002A13930690908C3E899400185
:100CFB001881D420650A08C3E899400281AD81D4DC
:100D0B00C265C2AF53E67F759100306712759400D0
:100D1B007595FE759104D26043E680D2AF81ADAE7E
:100D2B0040AF41C3E49EF594E49FF595A11EC3E546
:100D3B00339401500281AD30650281ADD802A14DD3
:100D4B0081D4C26DC2AF53E67F75910085539485F4
:100D5B005495759104854D92854E93D26043E680F0
:100D6B00D2AFE52D54066008206A020533020D8BC5
:100D7B00306D0D206C0A206507158115810215FB5E
:100D8B002278003064053065027801E53775F0078D
:100D9B00A4F9E5F028F5F0E9A2F013A2F113A2F201
:100DAB0013F537C394785003753778C3E537953807
:100DBB004008D266D297D295D293306002A1C585F6
:100DCB004F92855093D26043E68022207D16C2AFAE
:100DDB00754202C292D296306202C295D2AF759F13
:100DEB0013020FC5C2AF754202C292D29430620297
:100DFB00C297D2AF759F13020FC5307243207D206F
:100E0B00C2AF754203900134757B04D295C2943006
:100E1B006204C293C123D292D2AF759F10020FC549
:100E2B00C2AF754203900134757B04D297C29630E2
:100E3B006204C293C143D292D2AF759F11020FC508
:100E4B00207D17C2AF75420390010FD2953062021D
:100E5B00C293D2AF759F10020FC5C2AF75420390FC
:100E6B00010FD297306202C293D2AF759F11020F5E
:100E7B00C5207D16C2AF754204C296D29430620271
:100E8B00C293D2AF759F11020FC5C2AF754204C298
:100E9B0094D296306202C293D2AF759F10020FC5E7
:100EAB00307243207D20C2AF754205900123757BC4
:100EBB0040D293C292306204C297C1C9D296D2AFCC
:100ECB00759F13020FC5C2AF754205900145757B27
:100EDB0010D293C292306204C295C1E9D294D2AFC0
:100EEB00759F13020FC5207D17C2AF754205900188
:100EFB0005D293306202C297D2AF759F13020FC512
:100F0B00C2AF754205900119D2933062EBC295D2F4
:100F1B00AF759F13020FC5207D16C2AF754206C277
:100F2B0094D292306202C297D2AF759F10020FC556
:100F3B00C2AF754206C296D292306202C295D2AF50
:100F4B00759F11020FC5307243207D20C2AF7542D1
:100F5B0001900145757B10D297C296306204C29501
:100F6B00E16FD294D2AF759F11020FC5C2AF75421C
:100F7B0001900123757B40D295C294306204C297D5
:100F8B00E18FD296D2AF759F10020FC5207D17C28D
:100F9B00AF754201900119D297306202C295D2AF60
:100FAB00759F11020FC5C2AF754201900105D29515
:100FBB00306202C297D2AF759F10C26622900103B6
:100FCB00757B00D297D295D293C296C294C292C22D
:100FDB00622278807607087607087601087604087F
:100FEB0076FF0876FF08760B0876020876010876FE
:100FFB0001788C76010876000876B40876FF0876BF
:10100B00FF0876FF0876030876FF0876010876FF5F
:10101B000876250876D00876780876C8087604080E
:10102B0076FF08760108760008767A087607087648
:10103B00010876010876000876FF0876002278878B
:10104B00E6FFC2727888C27DE630E102D27DC27EB5
:10105B007889E630E102D27EC3EF94026008758E88
:0F106B0001D273021076758E00C273227880E670
:10107A00149000809378A5F67881E6149000809306
:10108A0078A6F67886E61490008D9378A7F6789F6E
:10109A00E6F8700108C3E8941140027811E828289C
:1010AA00F56B256B256B28F56C256B2828F56D7873
:1010BA0086E6F539C394025003753902789CE675C1
:1010CA0038FFB402037538A0B4030375388278A3D5
:1010DA00E61490009A93F566120FC822227896E6D3
:1010EA00FA7897E6FB7888E6B40305C3EB940EFB1F
:1010FA00307F047A007BFFC3EB9AFCC394825002D0
:10110A007C827572000572EC8572F0A4C3E5F094D6
:10111A007D40F222D27F11E71205527A007B007CD1
:10112A0010120548E55C2AFA74003BFBDCF37C04E8
:10113A00C3EB13FBEA13FADCF7FEC27F11E722E5E1
:10114A00EF20E6037520000520903FFFE52014609C
:10115A0006901DFF1460009304600375EF1253D9C3
:10116A00BF7581C043FF8012054375EF0243B20386
:10117A00E5B3240220E70DF521E5E320E006852109
:10118A00B343E301120FC87580FF75A40075F1B26D
:10119A0075D4DF7590A975A5FC75F2FE75D5017534
:1011AA00A60175E241120FC8E4F8F6D8FD75680188
:1011BA00120FDD12165278988673753001C2AF127B
:1011CA00055C12056C1205521205731205521205BE
:1011DA007A12055212177512055C12055C12055730
:1011EA00C2AF78FA79FA308507D9FBD8F7021C0022
:1011FA001149117711E611E778988673120FC875AD
:10120A00881075890275C82475910475D84075A827
:10121A002275B80275E690759B80759D0075D10E92
:10122A0075BC5875BB0875BA1175E880120543D2AA
:10123A00AF1208AB75360053DACF207E0343DA20AB
:10124A00307E0343DA1043DA01C2D8C27112055C58
:10125A00D2617B037A0CE55B70077A0CDB0302111F
:10126A00EA1205522070030211EAC270E55CC394C7
:10127A000240E1E52F541F855E5DF55EB55DD5DA66
:10128A00D5C26153DACF207E0343DA20307E03438E
:10129A00DA10C2D8C27178A2E67008D274E52F5467
:1012AA00E0F52FC275752900120557307409C3E598
:1012BA0029940A4002D275120548780230740278DD
:1012CA0000C3E55C9840F0C2AF12056C12056C12BF
:1012DA00056CD2AF12055C754C00120548788CE695
:1012EA00C3940150030213BAE530C39401500302B8
:1012FA0013BA207435C3E55C94FF50030213BAC2D3
:10130A00AF120581D2AF120557C3E55C940150EFC5
:10131A00C2AF12056C12054D12056CD2AF120557F9
:10132A00C3E55C94FF40E90217FA7F05D27F11E713
:10133A00120557C2AFC27F11E7AE5CC3E55C947F6A
:10134A00D2AF4076120543C2AF120581D2AFDFDCBD
:10135A00311EC3EE94057897F612055C12169412A4
:10136A00177D7F0AD27F11E7120557C2AFC27F11DC
:10137A00E7AE5CC3E55C947FD2AF50E6120543C288
:10138A00AF12056C12054D12056CD2AFDFD6311EB5
:10139A00EE24037896F612055C1216941217AC1214
:1013AA00055711E7C3E55C94FF500241FC0217FAA6
:1013BA00C3E55C954C4003855C4C1205577801796E
:1013CA0088E7B403027805C3E55C98400241E4C2A9
:1013DA00AF120581120581120581D2AF12055C7523
:1013EA003000E4F531F5320531E531F4703F05326C
:1013FA00789AE67819146012783214600D787D14A0
:10140A00600878FA146003753200C3E53298401D0B
:10141A00120FC8120543153275310078998673C2C6
:10142A00AF120581D2AF7898867312055712054D0F
:10143A00E52A700530740221EA78012074027806E0
:10144A00C3E55C9840A1120557E52A70030211EA28
:10145A00C2AF120FC8E4F522F523F524F525F526C7
:0E146A00F567D2AF7885E6C333F565E4F54447
:10147800F545F546F547F548F570F52CF52DF537A2
:1014880075700875BB1012054312093EE5E820EC9B
:10149800FBA8BDA9BEE97001F888711209427570F0
:1014A8000875BB101149C2AF7561FF1209FD85228D
:1014B80061852262852263D2AF7522017524017588
:1014C8002501752601856069756A017888E6B40387
:1014D80007C27D307602D27DD268D2697533001298
:1014E8000F22120F51120A1D120A24120A1D120A83
:1014F80024120A1D120C9F12065C120D8C120DD6B6
:10150800120A24120C8E306E031206FC2067031296
:10151800084E306703120895120D8C120E05120A38
:1015280024120C9F306E03120738120D8C120E7C99
:10153800120A24120C8E306E03120796120D8C12AA
:101548000EAB120A24120C9F306E031207F3120D11
:101558008C120F22120A2412093E120C8E120D8CC4
:10156800120F51120942120A2430692C85646185D0
:101578006462856069756A0179187A0CC3E53399E4
:101588004009C269D26A8A350215A0C3E55C940194
:1015980040030214FC021603306A1D206C1AE5355C
:1015A800147006C26AD26B81FCF535C3E55C940100
:1015B80040030214FC021603753600C3E55F94016C
:1015C8004009856462856069756A0178FA79A4E7DB
:1015D80060027803C3E55F985021307404E52A60FF
:1015E8001A78F0306C058564617820C3E54198501D
:1015F8000281FC0536E55C6002C106753600C2AFA3
:10160800120FC87887E6FE760211497887EEF6E46D
:10161800F522F523F524F525F526F565752C0075D5
:101628002D00D2AF120557120FC878A4E66006C283
:1016380097C293C295307406E52A700221EA788D24
:10164800E6C39401400241C161EC901A0D78201262
:1016580016D6E520B4A50CA31216D6E520B45A0375
:10166800021674120FDD121694021693901A03785C
:10167800807B0A1216D6A308DBF9901A0F788C7BA8
:10168800191216D6A308DBF9901A2822C2AF12172E
:10169800151216EF901A00740E1216DBA3740612B8
:1016A80016DBA374151216DB901A0378807B0A12D6
:1016B80016DAA308DBF9901A0F788C7B191216DA60
:1016C800A308DBF9121728121706901A2822E493A8
:1016D800F622E6438F01538FFD75EF0275B7A575A6
:1016E800B7F1F0538FFE22438F02438F0175EF024B
:1016F80075B7A575B7F1901A0DF0538FFC22901AA3
:101708000D74A5D1DB901A0E745AD1DB227A307988
:10171800D07820901A40D1D6E520F709A3DAF7222D
:101728007A3079D0901A40E7D1DB09A3DAF922ABF5
:1017380074A875BB01027980BB02027981BB0302E0
:101748007982BB04027994BB05027983BB060279CE
:1017580086BB07027992BB08027987BB0902799C8C
:10176800BB0A027988BB0B027989E8F7227C05124B
:10177800055CDCFB22C2AF12056C12057312057AF8
:1017880012058112054D12056C12057312057A12A5
:10179800058112054D12056C12057312057A1205A2
:1017A80081D2AF22C2AF12058112057A12057312D7
:1017B800056C12054D12058112057A120573120582
:1017C8006C12054D12058112057A12057312056C0B
:1017D800D2AF22AE74AF75C2AF12056C12056C128F
:1017E800056C12054DDEF212058112054DDFF8D2A7
:1017F800AF22F17DF1751217757574017575017554
:1018080076001217DB7C05AD5C12055CC3ED955CB8
:1018180070F5C3E55C9401400AC3E55C94FF40376A
:1018280002183C12173712169412177DC2AF75EFC3
:1018380012121775DCD10576C3E576940350028041
:10184800C11217750575E5741490009F93F808C3C5
:10185800E57598500280A81217751217750574C39C
:0E186800E574940C50028094120FDD12169459
:08187600C2AF75EF12121775E5
:0319FD000211498B
:101A00000E061507070104FFFF0B020101A55A018D
:101A100000B4FFFFFF03FF01FF25D078C804FF01DA
:091A200000FF07010100FF00FFB7
:101A4000235475726E696779364123202020202047
:101A500023424C48454C4923463333302320202031
:101A60002020202020202020202020202020202076
:101C0000C2AFC2D353D9BF7581C043B20343FF8073
:101C1000752438752503B1C975EF0275E24043F1AB
:101C20002053A4DF75D4FFD2857DFA780379E67C52
:101C300010752200752300901DD67B0675249875BB
:101C400025013085028142208508D8FBD9F9DCF7CF
:101C500081B4308508D8FBD9F9DCF781B4B189E4C7
:101C600093A3C39A6004DDC381B4DBDBB17B600264
:101C7000812B7B08E493FAA3B15CDBF87A30B15C8A
:101C8000752200752300B17BEAFCEBFDC3ED94FEE9
:101C9000400EB17B8A278B28ED30E0048A828B834B
:101CA000B17B7AC270D8C3ED94FE601350CEBD00F4
:101CB00025EC60097520007521FF0200008100A855
:101CC00027A9280809D804D90281D3B17FEA89AAB3
:101CD000F281C50D81A0C3ED94035049EDA2E092BD
:101CE000007AC5C3E5829400E583941C50902000DF
:101CF00010438F02438F0175B7A575B7F1F030001F
:101D00001FA827A9280809438F01538FFDD804D99C
:101D100002A12089AAE275B7A575B7F1F0A3A10DBC
:101D2000538FFC817C7AC1BD030CE493A3FAB140CC
:101D3000DCF8B138817C817EAA22AB23B15CEBFA5E
:101D4000EA6222752608C3E52313F523E52213F57D
:101D50002250066323A0632201D526EAB1C9B1C986
:101D600075260AEAF4200102D285300102C285B14B
:101D7000C9C3134002C201D526EB22B17FEAFB2082
:101D80008502A17F308502A184752608AE24AF2587
:101D9000C3EF13FFEE13FEB1CDB1C9C3EA13308513
:101DA000024480FA30E703632201C3E52313F523DD
:101DB000E52213F52250066323A0632201D526D91C
:101DC000E52265236523F52222AE24AF250E0FDE22
:101DD000FEDFFCD20122424C48656C693437316326
:041DE000F3300601D5
:00000001FF
